:10000000830100308A007328FC0003088301B200DA
:100010000408B3000A08B4008A017008BA007A081C
:10002000BB007B08BC003D08B9007108BE00720827
:10003000C5007308C6007408C4007508C0007608BF
:10004000BF007708C1007808C3007908C2003708EC
:10005000B5003808B600831206182F28302831283A
:10006000002883128619352836283E280D301521A0
:1000700039288312861D3D283E2839288312A2087C
:10008000031943284428472822081521A20180305B
:10009000831281000B1183123A08F0003B08FA002A
:1000A0003C08FB003908BD003E08F1004508F2009D
:1000B0004608F3004408F4004008F5003F08F60045
:1000C0004108F7004308F8004208F9003508B70076
:1000D0003608B8003308840034088A0032088300E8
:1000E000FC0E7C0E09002030840030308520830116
:1000F0000330B800FE30B700303084003230892041
:100100008301C12A04068001840A0406031D822893
:100110000034F00094208000840A0408700603195B
:1001200000348A288312B700B81B9D2838088A003B
:100130003708B70A0319B80A8200831338188317DF
:100140003708B70A840000080800203445344334D7
:1001500020344F344E34003420344534433420347A
:100160004F3446344634003434343834003439346F
:1001700036340034323434340034313439343234A7
:08018000003430343034003447
:10018A0083120513A5002508803E57218312080013
:10019A00831205130130572102303C2183120800D3
:1001AA00F400F40AF403031900340310F00DF10DFE
:1001BA00F20DF30DD728E228E22883128C1EE628D6
:1001CA00E728E12883121A08EA2883120800831212
:1001DA00981CF028F128F528181218160130F7286B
:1001EA000030F72883120800FB28FB2883128C1E94
:1001FA00FF280029FA28003083121819013005292E
:10020A00831208000929092983128C1E0D290E2937
:10021A0008290030831218180130132983120800A4
:10022A008312AF001929192983120C1E1D291E29B0
:10023A00182983122F089900222983120800831291
:10024A000517302983122508B8002408A40A0319BF
:10025A00A50A9220572183122508B8002408922063
:10026A000038031D39293A292729831208008312E5
:10027A00A60004308312A50053308312A700462932
:10028A0046298312A70B4A294B2945298312A50B14
:10029A004F29502941298312A60B542955293E2951
:1002AA00831208008312A600260E0F390F39F000B8
:1002BA000508F039700485008517851326080F395B
:1002CA00F0000508F03970048500851785130D3094
:1002DA00A700702970298312A70B742975296F2921
:1002EA008312080083120517A500250E0F390F394E
:1002FA00F0000508F0397004850085178513250874
:10030A000F39F0000508F039700485008517851348
:10031A000D30A600912991298312A60B95299629B9
:10032A00902983120800831205130F303C210330F1
:10033A0085008517851305303C21851785132130E3
:10034A00A400A829A8298312A40BAC29AD29A7299E
:10035A0083128517851305303C21023085008517E5
:10036A0085130D30A400BA29BA298312A40BBE2919
:10037A00BF29B92928305721083057210F30572172
:10038A0006305721831208008312A4000C3024027D
:10039A000318D029DC290E302402031CDB29D529B5
:1003AA00203024020318DB29DA29DC29DD29DF2998
:1003BA00DE29E0291A2AFD29CD20A101062A1130B9
:1003CA00831221020318EA29EB29EE294030A10001
:1003DA00F6295130831221020318F429F529F62946
:1003EA00A101062A831224087721A10A062A062ACD
:0603FA00831224080C3AF6
:100400000319E129013A0319E429F7298312210884
:10041000103A031D0C2A0D2A0F2A4030A100831226
:100420002108503A031D152A162A172AA101831202
:100430002108C5208312080083122408F000250833
:10044000F1002608F2002708F3000430D5207008D8
:10045000AB007108AC007208AD007308AE002B0849
:10046000F4002C08F5002D08F6002E08F7000030E7
:10047000F0000930F1003D30F2000030F300742349
:10048000FF307007A900FF30031800307107AA0081
:100490002A08803AF00081307002003003192902E6
:1004A000031C532A562AAA1F572A562A592A582A61
:1004B0009B2A2408F0002508F1002608F2002708EE
:1004C000F3000630D5207008AB007108AC0072084C
:1004D000AD007308AE002B08F4002C08F5002D08C1
:1004E000F6002E08F7000030F0000930F1003D3032
:1004F000F2000030F3007423FF307007A900FF30D2
:10050000031800307107AA002A08803AF0008130F1
:100510007002003003192902031C8F2A922AAA1F95
:10052000932A922A952A942A982A0130BF2A9A2A35
:10053000831618119D2A831618158312290883160D
:1005400099001812831298171816981283160C1215
:100550008C128312A808031DAE2AB12A831618171D
:10056000B32A831618138312A808031DB82ABA2ABF
:100570001817BB2A1813831698160030BF2A831247
:100580000800303083168500FB3086008312850119
:10059000860107309F00831681018B138B128030F8
:1005A000831281008B170B179821CD20861BD92A27
:1005B000DA2A3A2B042B60308312B0000930B100E4
:1005C000BA30A4000030A50024211B2BC0308312B8
:1005D000B0001230B100B430A4000030A5002421D6
:1005E0001B2B80308312B0002530B100B730A4003F
:1005F0000030A50024211B2BBD308312A400003045
:10060000A50024211B2B1B2B8312060E0F39033947
:10061000F200F301162B7208013A0319F12A033A8A
:100620000319E62A013A0319DB2AFC2A7308003A67
:1006300003190B2BFC2AC1308312A4000030A50043
:1006400024210030061B0130A000A0080319292B2B
:100650002A2B302BAC30A4000030A5002421362BEF
:10066000A5308312A4000030A50024214030C5200D
:100670004030A10083123008F0003108F100003052
:10068000F11BFF30F200F3007008A4007108A50010
:100690007208A6007308A700A8011C224F2B831222
:1006A000061C532B542B4F2B8B16722BE020A300D0
:1006B0002308C921A008031D5E2B5F2B612B230893
:1006C000A200EC2000380319662B672B722B682BD5
:1006D0008316981C6C2B6D2B682B831218123F30DD
:1006E000A2001816562B732884018312BD01F8014D
:1006F000F901FA01FB017408750476047704031903
:10070000842BC030BD058F2BF001F101F201F30104
:10071000EF2B0310F40DF50DF60DF70DBD0AF71FC5
:10072000892BBD0A0310F80DF90DFA0DFB0D7708A2
:100730007302031DA52B76087202031DA52B7508F5
:100740007102031DA52B74087002031CB72B7814CB
:100750007408F0027508031C750FF1027608031C7B
:10076000760FF2027708031C770FF3020310F70CE1
:10077000F60CF50CF40CBD033D083F39031D922B1C
:100780003D1FCF2B0310FF30F007F009031CF107CA
:10079000F109031CF207F209031CF307F3097008BF
:1007A000F4007108F5007208F6007308F700780885
:1007B000F0007908F1007A08F2007B08F300BD1F11
:1007C000EF2B0310FF30F007F009031CF107F109CC
:1007D000031CF207F209031CF307F309EF2B84084B
:1007E00003190034730880008403720880008403B6
:1007F00071088000840370088000003400344B349A
:02400E00503F21
:00000001FF
